:020000040000FA
:10002000831603138501FF30860003308700831297
:100030008A01A801A701A601A501A401A301A201AB
:10004000A101A00190019015901487116430AC00BB
:10005000A80107158E018F01071110148715502074
:10006000AC0B2F281E30AB00AB0B342887111010BF
:100070000330AC005020AC0B3A28A701A601A50123
:10008000A401A301A201A101A0010F08B2006B20ED
:100090000E08B2006B200608B2006B208D202628C7
:1000A0000708F0388700280A0739A8008500203E95
:1000B0008400000EF039A90007080C3929048700D4
:1000C000C830AB00AB0B622800007C30AB00AB0B40
:1000D000672800000800B301B601B401B501B21BE6
:1000E000B40A3508203E84000310800D3418800ABD
:1000F0000008063EB300B401331E8128B40A0A305A
:100100008002B50A07303502031D7128B60A08308F
:10011000360203190800B20D6D28A608031D080059
:100120000F30A600A508031D08000F30A500A40885
:10013000031D08000F30A400A308031D08000F30A2
:04014000A300080010
:02400E00793FF8
:00000001FF
